:020000040000FA
:10420000480065006C006C006F00200049005200FF
:1042100044004100200062006F0061007200000055
:104220005000610075006C0066006A0075006A004D
:104230006F0040006600720065006500000000002D
:104240003100360046003800370037005F00490073
:1042500072006400610062006F006100720064001F
:104260005F0046006C006F00610074005F004C004E
:10427000430044005F00520053005F00500069009B
:10428000630045004500700072006F006D005F0024
:10429000320034004C0043003200350036005F002D
:1042A0004400530031003300300037005F0031001C
:1042B000340030003600300033002E006300000070
:1042C0004D00430050003200310035003000200026
:1042D000440069007300610062006C0065006400C6
:1042E0002000420079002000520065007300650044
:1042F000740020000D000A00000000000000000013
:10430000FF00FF00FF00FF00FF00FF00FF00FF00B5
:10431000FF00FF00FF00FF00FF00FF00FF00FF00A5
:10432000FF00FF00FF00FF00FF00FF00FF00FF0095
:10433000FF00FF00FF00FF00FF00FF00FF00FF0085
:104340004D0069006B0072006F00430020003100D7
:104350003600460038003700370020004900520080
:1043600044004100200062006F00610072006400A0
:1043700020005400650073007400200050004900C4
:104380004300200045004500500052004F004D0002
:104390002000310039002D00300031002D003200A6
:1043A00030003100340020000D000A000000000041
:1043B00000000000000000000000000000000000FD
:1043C0007000610075006C0066006A0075006A008C
:1043D0006F00400066007200650065002E006600F8
:1043E00072000D000A000000FF00FF00FF00FF0048
:1043F000FF00FF00FF00FF00FF00FF00FF00FF00C5
:00000001FF
